:100000000C94A5050C94DD050C94DD050C94DD0520
:100010000C94DD050C94DD050C94DD050C94DD05D8
:100020000C94DD050C94DD050C944F2A0C94212BC7
:100030000C9485240C94DD050C94DD050C94DD05F1
:100040000C94DD050C94DD050C94DD050C94DD05A8
:100050000C94DD050C940D250C94DD050C94DD0548
:100060000C94DD050C94DD050C94DD050C94DD0588
:100070000C94DD050C94DD050C94DD050C94DD0578
:100080000C94DD050C94DD050C94DD050C94DD0568
:100090000C94DD050C94DD050C94DD050C94DD0558
:1000A0000C94DD050C94DD050C94DD05910A910A94
:1000B000BD0ABD0A250B430B5B0C5B0C4E0BE70B1B
:1000C000F80BF80B8E2BB52BAD2CB52BAD2C012CD2
:1000D000242CAD2C7B2C8A2C68747470733A2F2FCF
:1000E000716D6B2E666D2F01012800514D4B2069FB
:1000F00073207468652062657374207468696E6724
:100100002065766572210027001E001F0020002157
:1001100000220023002400250044454255473A2090
:1001200064697361626C65642E0A004445425547F8
:100130003A20656E61626C65642E0A000000000062
:10014000000000002A2B2800000000000000000032
:100150000000000000000029000000002C1E3420D8
:10016000212224342627252E362D3738271E1F20FE
:100170002122232425263333362E37381F04050643
:100180000708090A0B0C0D0E0F1011121314151687
:100190001718191A1B1C1D2F3130232D3504050685
:1001A0000708090A0B0C0D0E0F1011121314151667
:1001B0001718191A1B1C1D2F3130354C0000000078
:1001C000000000000000000000000000000000002F
:1001D000000000000000000000000000000000001F
:1001E0007E0F00D4FFFFFFC7000000780A00253013
:1001F0003258006C65645F7461736B3A20004F6E17
:100200006573686F743A206163746976653A202576
:10021000640A000A0025303862003A200025303296
:1002200058000A722F632030313233343536370AA2
:1002300000290A002575002F002575005D2800257E
:10024000640020002564002000256400200025644F
:10025000007C0025303258006D6F7573656B6579D1
:10026000205B62746E7C782079207620685D28722D
:1002700065702F61636C293A205B006261636B6C6F
:100280006967687420737465703A2025750A006286
:1002900061636B6C696768742064697361626C6523
:1002A0000A006261636B6C6967687420656E6162E5
:1002B0006C650A006261636B6C6967687420746FB7
:1002C00067676C653A2025750A006261636B6C692B
:1002D0006768742064656372656173653A2025758B
:1002E0000A006261636B6C6967687420696E63728F
:1002F000656173653A2025750A00313A0964656CB9
:100300006179282A31306D73293A2025750A323AED
:1003100009696E74657276616C286D73293A2025BF
:10032000750A333A096D61785F73706565643A20C8
:1003300025750A343A0974696D655F746F5F6D6184
:10034000783A2025750A353A09776865656C5F6DDE
:1003500061785F73706565643A2025750A363A09DD
:10036000776865656C5F74696D655F746F5F6D61FB
:10037000783A2025750A00703A097072696E742007
:1003800076616C7565730A643A09736574206465F7
:100390006661756C74730A75703A092B310A646E64
:1003A0003A092D310A6C743A092B31300A72743AC9
:1003B000092D31300A4553432F713A09717569741B
:1003C0000A0A7370656564203D2064656C74612061
:1003D0002A206D61785F7370656564202A20287219
:1003E0006570656174202F2074696D655F746F5F3F
:1003F0006D6178290A77686572652064656C74613F
:100400003A20637572736F723D25642C207768659E
:10041000656C3D25640A53656520687474703A2FD5
:100420002F656E2E77696B6970656469612E6F72D6
:10043000672F77696B692F4D6F7573655F6B657992
:10044000730A004D3E20004D25753A25733E20006D
:100450003F0A003D2025750A003F0A006465666179
:10046000756C74730A0025750A003F0A000A092D8D
:100470002056616C756573202D0A00710A000A0907
:100480002D204D6F7573656B6579202D0A003F0037
:10049000433E20004C25640A000A092D2053746154
:1004A000747573202D0A686F73745F6B6579626F62
:1004B0006172645F6C65647328293A202530325874
:1004C0000A6B6579626F6172645F70726F746F63DB
:1004D0006F6C3A20253032580A6B6579626F617211
:1004E000645F69646C653A20253032580A74696D1E
:1004F00065725F72656164333228293A202530388D
:100500006C580A000A092D2056657273696F6E20B7
:100510002D0A5649443A20307846454544285472BD
:1005200065617375726529205049443A20307830EE
:100530003030302854797065203929205645523A98
:10054000203078303030310A4255494C443A20202E
:10055000284665622032382032303232290A4F5024
:1005600054494F4E533A204C554641204D4F555318
:10057000454B45592045585452414B455920434F0E
:100580004E534F4C4520434F4D4D414E4420343047
:1005900039360A4743433A20352E342E302041560F
:1005A000522D4C4942433A20322E302E30204156B3
:1005B000525F415243483A20617672350A000A0977
:1005C0002D20436F6E736F6C65202D0A4553432FAA
:1005D000713A09717569740A6D3A096D6F757365C1
:1005E0006B65790A000A092D204D61676963202D2A
:1005F0000A443A094465627567204D657373616703
:100600006520546F67676C650A583A094D617472CA
:100610006978204465627567204D6F646520546F6A
:1006200067676C65202D2053686F77206B65797044
:1006300072657373657320696E206D617472697879
:1006400020677269640A4B3A094B6579626F61727F
:100650006420446562756720546F67676C65202D60
:100660002053686F77206B657970726573732072A1
:1006700065706F72740A4D3A094465627567204D62
:100680006F75736520546F67676C650A563A095633
:10069000657273696F6E0A533A09537461747573A6
:1006A0000A433A09416374697661746520436F6E49
:1006B000736F6C65204D6F64650A46312D4631308D
:1006C0003A0953776974636820746F204C617965C7
:1006D0007220302D392028463130203D204C3029E1
:1006E0000A302D393A0953776974636820746F2092
:1006F0004C6179657220302D390A47524156453A8E
:100700000953776974636820746F204C617965724E
:1007100020302028616C7465726E617465290A420C
:100720003A094A756D7020746F20426F6F746C6F58
:10073000616465720A4553433A094A756D702074C5
:100740006F20426F6F746C6F616465722028616CFA
:100750007465726E617465290A453A095072696E52
:100760007420454550524F4D2053657474696E672F
:10077000730A4253504143453A09436C6561722004
:10078000454550524F4D0A006261636B6C69676862
:10079000745F636F6E6669672E7261773A202530E9
:1007A00032580A2E656E61626C653A2025750A2EF4
:1007B0006C6576656C3A2025750A006B65796D610C
:1007C000705F636F6E6669672E7261773A202530BD
:1007D00032580A2E737761705F636F6E74726F6C3C
:1007E0005F636170736C6F636B3A2025750A2E63CB
:1007F0006170736C6F636B5F746F5F636F6E747245
:100800006F6C3A2025750A2E737761705F6C637484
:100810006C5F6C6775693A2025750A2E7377617075
:100820005F7263746C5F726775693A2025750A2E72
:10083000737761705F6C616C745F6C6775693A2087
:1008400025750A2E737761705F72616C745F7267D1
:1008500075693A2025750A2E6E6F5F6775693A20B3
:1008600025750A2E737761705F67726176655F65C3
:1008700073633A2025750A2E737761705F62616336
:100880006B736C6173685F6261636B7370616365E6
:100890003A2025750A2E6E6B726F3A2025750A0074
:1008A00064656275675F636F6E6669672E726177F4
:1008B0003A20253032580A2E656E61626C653A2006
:1008C00025750A2E6D61747269783A2025750A2E95
:1008D0006B6579626F6172643A2025750A2E6D6FBF
:1008E0007573653A2025750A006565636F6E6669E4
:1008F000673A0A64656661756C745F6C61796572EC
:100900003A2025750A003F000A6D6F7573653A201D
:100910006F66660A000A6D6F7573653A206F6E0A1E
:10092000000A6B6579626F6172643A206F66660ACD
:10093000000A6B6579626F6172643A206F6E0A001B
:100940000A6D61747269783A206F66660A000A6DF2
:1009500061747269783A206F6E0A000A6465627584
:10096000673A206F66660A000A64656275673A2016
:100970006F6E0A000A0A4A756D70696E6720746F9F
:1009800020626F6F746C6F616465722E2E2E200072
:10099000433E2000436C656172696E672045455097
:1009A000524F4D0A000A002530325820006B6579FD
:1009B000626F6172645F7265706F72743A20005B7F
:1009C000735D005B575D005B535D005B525D005BD8
:1009D000445D005B435D000E0354007900700065C8
:1009E000002000390000001203540072006500610D
:1009F000007300750072006500000004030904091B
:100A0000025B00030100A0FA0904000001030101D8
:100A1000000921110100012240000705810308009F
:100A20000109040100010300000009211101000176
:100A3000227B000705820320000109040200020353
:100A40000000000921110100012222000705830393
:100A5000200001070503032000011201000200002D
:100A60000008EDFE00000100010200010631FF094F
:100A700074A1010975150026FF00952075088102F3
:100A80000976150026FF00952075089102C0050122
:100A90000902A10185020901A1000509190129081E
:100AA00015002501950875018102050109300931FC
:100AB0001581257F95027508810609381581257FE6
:100AC000950175088106050C0A38021581257F9568
:100AD0000175088106C0C005010980A101850319BF
:100AE000012AB700150126B700950175108100C0D5
:100AF000050C0901A101850419012AA0021501268E
:100B0000A002950175108100C005010906A101052B
:100B10000719E029E715002501950875018102955F
:100B200001750881010507190029FF150026FF003E
:100B300095067508810005081901290595057501B7
:100B40009102950175039101C00011241FBECFEFE2
:100B5000DAE0DEBFCDBF04B603FE18C08091A80264
:100B60009091A902A091AA02B091AB028730904B5C
:100B7000A740B04B59F41092A8021092A90210920B
:100B8000AA021092AB02E0E0F8E3099511E0A0E0C0
:100B9000B1E0EEE6FBE502C005900D92AE3EB10776
:100BA000D9F722E0AEEEB1E001C01D92A83AB2073B
:100BB000E1F70E946D180C94B52D0C940000FF9382
:100BC000EF93E091EE01F091EF01309709F0099574
:100BD000EF91FF910895FC018591803011F0EFDFD6
:100BE000FBCF0895FF27E0E230E247FF0CC04195BC
:100BF00097FF09C0EDE26095709580959095611D15
:100C0000711D811D911D27FF02C0219530E350E227
:100C1000AA27660F771F881F991FAA1FA41710F015
:100C2000A41B63955A95A9F7AA3008F0A95FA05DA7
:100C3000AF93F395611571058105910541F7ED328B
:100C400011F4EF93F395F21718F43F93F395FBCF5C
:100C50008F91B5DFFA95E1F70895E991F9918591C2
:100C6000803021F0853219F0AADFF9CF089520E015
:100C7000E89455915532C1F3503311F4689455916D
:100C80005A3348F4505390F3220F022E220F220FB2
:100C9000200D250FF4CF0EF42195899199915336AB
:100CA00019F3533729F1533559F1BC018827992796
:100CB000E8945C3621F48991999168945591543661
:100CC00039F446EF7EF077FF0DC08FEF9FEF0AC03B
:100CD00055374AE039F0583540E121F0523642E0CC
:100CE00009F00895FF93EF937DDFEF91FF91B7CF68
:100CF000FF93EF93FC0181918030B9F360DFFBCF6C
:100D0000FF93EF9368DFF1CFDF93CF93CDB7DEB7DB
:100D10002596A3DFCF91DF910895873A2DE59207BD
:100D200021F0883A9D4541F00FC0FB018281882364
:100D300059F08BEE90E006C0FB018281882321F000
:100D400088ED90E00E94620881E0089581E00895B6
:100D50000C948D0608950C94AA061F93CF93DF93ED
:100D600000D000D01F92CDB7DEB749835A836B8382
:100D70003091F10189819A81311114C0662359F0B3
:100D8000222349F00E94980E182F682F89819A819A
:100D90000E94410E03C00E946C0E182F69817A8157
:100DA000812F04C00E94980E69817A810F900F9064
:100DB0000F900F900F90DF91CF911F910C94CD1554
:100DC000FC01262F408151816281738184810C94C2
:100DD000AD0681E00895CF93DF93EC0160E00E94BF
:100DE000E006BE01DF91CF910C94AB060C943F1747
:100DF0000C943B1708950E94EB0C0E94FA062FEF0B
:100E000084E39CE0215080409040E1F700C0000066
:100E10000C9433250F931F93CF93DF938C0161E0E4
:100E20000E94E006EC01B8010E94A806882309F49C
:100E300062C0B801CE010E94DE1C882309F45BC0A9
:100E4000B801CE010E941323882309F454C0B801CD
:100E5000CE010E94D91D882309F44DC0B801CE01EE
:100E60000E946F22882309F446C0F80182818823FA
:100E7000D9F1CF3D8CE5D80779F140F4C115FCE5F7
:100E8000DF0791F0C130DC4591F02EC0CC35EDE5A7
:100E9000DE0741F1CD35FDE5DF0709F1CB35DD4555
:100EA00019F50E942F1320C00E94FB0624C08091D8
:100EB0005B02C82FC095C170C0FB80F980935B02B4
:100EC000CC2329F08BE291E00E94EB0514C089E16C
:100ED00091E00E94EB0510C00E94DD130CC00E943F
:100EE000261302C00E943213C801DF91CF911F91D7
:100EF0000F910C94A606C0E08C2FDF91CF911F912B
:100F00000F9108950E94682480E00E94131D0C94A4
:100F100088080E94961B0E948B080C946E24DF9216
:100F2000EF92FF920F931F93CF93DF93E82FF0E0A0
:100F3000E45CFE4FD490282F26952695269530E028
:100F4000F901E452FE4F0491877010E0082E02C0B0
:100F5000159507950A94E2F701701127F901E453FA
:100F6000FE4FE490F12C082E02C0F594E7940A9409
:100F7000E2F791E0E922FF24F901E454FE4FC49125
:100F8000D0E002C0D595C7958A95E2F7C170DD27FC
:100F90000115110519F081EE0E941109E114F10407
:100FA00019F086EE0E9411098D2D0E943F0AEF284C
:100FB00019F086EE0E94C009012B19F081EE0E9403
:100FC000C009CD2B51F08CE2DF91CF911F910F9191
:100FD000FF90EF90DF900C943F0ADF91CF911F912B
:100FE0000F91FF90EF90DF900895EF92FF920F9393
:100FF0001F93CF93DF938C01F62E8AE0E82EF80141
:101000008491882309F457C0813009F042C0E80177
:101010002196FE018491813031F42196FE01849164
:101020000E943F0A39C0823039F4E8012296FE015D
:1010300084910E94110930C0833039F4E80122966E
:10104000FE0184910E94C00927C0843029F5E8017F
:101050002296FE01249180E090E030E02053310997
:101060002A30310560F4E89EA001E99E500D11245C
:10107000C901840F951F2196FE012491EECF0097A0
:1010800059F0EFE9FFE03197F1F700C00000019758
:10109000F6CF0E948F07E8018E010F5F1F4F8F2D43
:1010A000882309F4ACCFEFE9FFE03197F1F700C0F6
:1010B00000008150F5CFDF91CF911F910F91FF90EC
:1010C000EF90089560E00C94F5078295982F937344
:1010D00044E0949F900111248C7C86958695282B62
:1010E000822F8575880F2A7A2695822B0895089578
:1010F0000C94770881E008950C947A080895CF93B2
:10110000C82F0E9478088C2F0E947C08CF910895E8
:1011100080E00C947F080E946F230C947F08CF938B
:101120000E946F23C82F8091F001C81741F1C0932E
:10113000F00180915B0282FF1EC080FF04C083EF3C
:1011400091E00E94EB0580915B0280FF0CC01F9232
:10115000CF938EEE91E09F938F930E9484060F9021
:101160000F900F900F9080915B0280FF04C08CEE77
:1011700091E00E94EB058C2FCF910C947F08CF91CA
:101180000895CF93DF93CDB7DEB72B970FB6F894C2
:10119000DEBF0FBECDBF4F83588769877A878B87A5
:1011A00061110E945E129E012F5F3F4F86E0F901A0
:1011B00011928A95E9F785E0FE013796D9010190F1
:1011C0000D928A95E1F789819A814C815D81452B49
:1011D00031F09F3F31F491E08F3F19F403C091E06B
:1011E00001C090E090FF09C049815A816B817C81E8
:1011F0008D819E810E947F1105C0C9010E94E90670
:101200008111F2CF2B960FB6F894DEBF0FBECDBF83
:10121000DF91CF910895FC01808191810E94DA0EC7
:101220000895CF93882309F4A9C0C82F8238C1F448
:101230000E946F2381FDA2C069E380910201909119
:1012400003010E9440240E9480122FEF81EE94E05F
:10125000215080409040E1F700C0000069E319C0D0
:10126000833801F50E946F2380FD88C063E580917B
:101270000201909103010E9440240E9480122FEFEE
:1012800081EE94E0215080409040E1F700C00000E2
:1012900063E580910201909103010E944224CF9165
:1012A0000C9480128438C1F40E946F2382FD66C0C2
:1012B00067E480910201909103010E9440240E9402
:1012C00080122FEF81EE94E0215080409040E1F7B2
:1012D00000C0000067E4DDCF8CEF8C0F813AF8F49A
:1012E0008C2F0E941822811149C06C2F809102011D
:1012F000909103010E940A24882349F06C2F809169
:101300000201909103010E9442240E9480126C2FDE
:1013100080910201909103010E944024C0CF80E29D
:101320008C0F883048F4C77081E001C0880FCA95DF
:10133000EAF70E944112B3CFEBE5EC0FE33040F443
:10134000F0E0E95BFE4F808190E0CF910C94D223D6
:10135000E8E5EC0FE73150F4F0E0EE0FFF1FE75E39
:10136000FE4F80819181CF910C94E823CD3E30F0E7
:101370008C2F0E94F218CF910C94C419CF9108952C
:10138000882309F464C0823879F40E946F2381FFB6
:101390005EC069E380910201909103010E944024A4
:1013A0000E94801269E310C08338B1F40E946F2359
:1013B00080FF4DC063E580910201909103010E947E
:1013C00040240E94801263E5809102019091030104
:1013D0000E9442240C948012843879F40E946F2376
:1013E00082FF35C067E480910201909103010E9461
:1013F00040240E94801267E4E7CF9CEF980F913A57
:1014000010F4682FE1CF90E2980F983050F4877075
:1014100091E001C0990F8A95EAF7892F0E9447123F
:10142000D9CF9BE5980F933020F480E090E00C94A6
:10143000D22398E5980F973120F480E090E00C9447
:10144000E8238D3E20F00E944D190C94C419089594
:101450001F93CF93DF93182FEB010E941109209760
:1014600041F08FE99FE00197F1F700C0000021975C
:10147000F6CF812FDF91CF911F910C94C009893352
:1014800019F060E070E002C060E570E00C94280A9A
:10149000882321F00E9441120C9480120895882321
:1014A00021F00E9447120C9480120895CF92DF928F
:1014B000EF92FF920F931F93CF93DF937C01D62F70
:1014C000C72FFC011281058102950F700E9437120F
:1014D0008823B9F01123A9F08C2F807F803421F06C
:1014E00080E28D0F883068F080918F0282FD09C004
:1014F00082E00E94E0120E94371291E0D82ED92695
:1015000001C0D12CCC2EC2948FE0C8228C2D90E04B
:101510008C30910508F0CFC1FC01EA5AFF4F0C94C2
:10152000462D8C2F807FCF70882311F0C295C07F0D
:10153000112399F0CC2309F4AAC180E28D0F8830E1
:1015400010F0D11104C08C2F0E94411203C08C2FC7
:101550000E9451120E9480129AC18D2F0E94C009D0
:10156000CC2309F4A8C180E28D0F883038F1DD2347
:1015700029F18C2F0E94571224C08C2F807FCF70AE
:10158000803211F0C295C07FDD2319F0D130A1F176
:101590003DC080918F0282FF17C0112349F0CC23F8
:1015A00029F08C2F0E9441120E94801280E070C1AD
:1015B00080E00E94C009CC2309F47DC18C2F0E94D9
:1015C00047120E94801277C1112371F0002341F06D
:1015D000013031F40E9461128C2B0E9469126BC1A0
:1015E0000E9461128C2B1DC0002319F0013009F4F8
:1015F00062C10E94761225C0112321F0063008F046
:101600005AC10EC0053008F056C11BC0112361F04D
:10161000002331F0F701858180FF39C18F70858308
:101620008C2F0E94480A47C1002359F0D93309F092
:101630003FC1FFEF07EE13E0F15000401040E1F72B
:1016400035C18C2F0E944F0A36C18C2F8695869506
:10165000837019F0813061F02EC1112321F08D2F9C
:101660009C2F937002C080E090E00E94D2232BC197
:10167000112321F08D2F9C2F937002C080E090E009
:101680000E94E82320C18D2F112319F00E94F21827
:1016900002C00E944D190E94C41915C18C2F83707D
:1016A00009F047C011110BC12D2F229526952770E7
:1016B000220F220F6D2F6F70862F90E0A0E0B0E018
:1016C000022E04C0880F991FAA1FBB1F0A94D2F7CD
:1016D000D4FF10C04FE050E060E070E004C0440F61
:1016E000551F661F771F2A95D2F740955095609534
:1016F000709503C040E050E0BA01C695C695C3702E
:101700008A019B01082B192B2A2B3B2BC901B801FD
:10171000C23049F058F4C13019F00E94570DCFC0C3
:101720000E94450DCCC00E94690DC9C00E94430DA6
:10173000C6C0112319F08C2F817001C086958823B3
:1017400009F4BDC02D2F229526952770220F220F58
:101750006D2F6F70862F90E0A0E0B0E0022E04C0E5
:10176000880F991FAA1FBB1F0A94D2F7D4FF10C07D
:101770004FE050E060E070E004C0440F551F661F6A
:10178000771F2A95D2F7409550956095709503C0C4
:1017900040E050E0BA01C695C695C3708A019B012E
:1017A000082B192B2A2B3B2BC901B801C23049F059
:1017B00058F4C13019F00E941C0E81C00E940A0E1C
:1017C0007EC00E942E0E7BC00E947D0D78C0CF701F
:1017D000112339F08C2F0E94A30D8D2F0E94480AEF
:1017E0006EC08D2F0E944F0A8C2F0E94C40D67C0BF
:1017F000D23F21F128F4D03F41F0D13FC1F043C0A6
:10180000D33F19F1D43F79F03EC0112341F00530A8
:1018100008F051C08C2F8F710E94E90D4CC006302A
:1018200008F049C0F7CF80918F0282FF18C01123C2
:1018300039F08C2F8F710E94A30D3DC01123C9F385
:101840008C2F8F710E94C40D36C0112329F08C2F6C
:101850008F710E948E0D2FC00E94890D2CC0112304
:1018600049F0CF718C2F0E94A30D63E08C2F0E9452
:10187000C51221C081E00E94E0120230E0F082E057
:101880000E94E01218C0112331F0002391F28D2F35
:101890000E94110910C0002399F2D93349F41FEFB7
:1018A00027EE33E0115020403040E1F700C0000047
:1018B0008D2F0E94C00988EF8C0D843020F40E9487
:1018C0006F230E947F08DD20C9F00E94331280FD43
:1018D00015C0F70112820E942D120E94A30DC701AC
:1018E0000E949F0C0E942D12DF91CF911F910F91AA
:1018F000FF90EF90DF90CF900C94C40DDF91CF91CB
:101900001F910F91FF90EF90DF90CF9008950F936C
:101910001F93CF93DF93EC01688179818A810E94C4
:10192000E50E8C010E94400E0E94310DB801CE01DF
:101930000E94560ADF91CF911F910F910895CF9386
:10194000DF93EC01988189812B813C81232B31F03D
:101950008F3F31F481E09F3F19F403C081E001C063
:1019600080E080FD1DC0CE010E940A07811110C0D9
:101970000E9437128823A1F08A81882389F0809100
:101980008F0282FD0DC082E0DF91CF910C94E012B6
:10199000CE010E94870CCE01DF91CF910C94EB0613
:1019A000DF91CF91089580E090E00E94D22380E003
:1019B00090E00E94E8230E945E120E9480120E9422
:1019C000771B0C94C41980910201909103010E942D
:1019D00044240C94D30C0E944E120C94E30C929568
:1019E0009F70963079F010F4925001C09A50923066
:1019F00068F4803F69F018F4883E40F409C0843FE1
:101A000029F406C0883E20F0813F11F080E008955F
:101A100081E00895FC01808191810E94DA0E0E948C
:101A2000EF0C0895CF93DF9300D000D01F92CDB775
:101A3000DEB70F900F900F900F900F90DF91CF9126
:101A40000895CF93DF9300D000D000D0CDB7DEB79C
:101A500026960FB6F894DEBF0FBECDBFDF91CF91B3
:101A60000895089508950C94320D0C94330D0E943E
:101A7000350D6093000270930102809302029093EF
:101A800003020C94D30C0C94370D0F931F93009109
:101A90000002109101022091020230910302602B9A
:101AA000712B822B932B1F910F910C94370D0F9359
:101AB0001F930091000210910102209102023091C7
:101AC000030260237123822393231F910F910C94AF
:101AD000370D0F931F930091000210910102209186
:101AE00002023091030260277127822793271F91FA
:101AF0000F910C94370D0C94320D0E947B0D609366
:101B0000FC017093FD018093FE019093FF010C9402
:101B1000D30C60E070E0CB010C947D0D0F931F930C
:101B200041E050E060E070E08A019B0104C0000FDA
:101B3000111F221F331F8A95D2F7C901B8011F91C7
:101B40000F910C947D0D0F931F9341E050E060E0E6
:101B500070E004C0440F551F661F771F8A95D2F7A7
:101B60008091FC019091FD01A091FE01B091FF01D7
:101B70008A019B01082B192B2A2B3B2BC901B80189
:101B80001F910F910C947D0D0F931F9341E050E036
:101B900060E070E004C0440F551F661F771F8A95F0
:101BA000D2F740955095609570958091FC01909189
:101BB000FD01A091FE01B091FF018A019B01082364
:101BC00019232A233B23C901B8011F910F910C94BB
:101BD0007D0D0F931F9341E050E060E070E004C082
:101BE000440F551F661F771F8A95D2F78091FC011D
:101BF0009091FD01A091FE01B091FF018A019B012E
:101C0000082719272A273B27C901B8011F910F91DF
:101C10000C947D0D0F931F930091FC011091FD0119
:101C20002091FE013091FF01602B712B822B932BB1
:101C30001F910F910C947D0D0F931F930091FC0148
:101C40001091FD012091FE013091FF01602371236D
:101C5000822393231F910F910C947D0D0F931F935B
:101C60000091FC011091FD012091FE013091FF01D6
:101C700060277127822793271F910F910C947D0D68
:101C80000895292F220F920F890FE82FE695E695E8
:101C9000E695877051E001C0550F8A95EAF785E017
:101CA000E89FF0011124EE50FE4F20E030E070E09C
:101CB0004081CB01022E02C0969587950A94E2F7E7
:101CC0008170819584278523842781932F5F3F4FDF
:101CD0002530310569F70895292F220F920F890FBA
:101CE000682F669566956695982F977085E0689F32
:101CF000B001112440E050E080E0FB01E40FF51F4B
:101D0000EE50FE4F208130E0092E02C03695279517
:101D10000A94E2F721703327042E01C0220F0A949F
:101D2000EAF7822B4F5F5F4F4530510531F7089539
:101D3000BF92CF92DF92EF92FF920F931F93CF93B8
:101D4000DF938C01C090FC01D090FD01E090FE017A
:101D5000F090FF018091000290910102A091020297
:101D6000B0910302C82AD92AEA2AFB2ACFE1D0E09F
:101D7000D701C6010C2E04C0B695A79597958795F7
:101D80000A94D2F780FD04C0219790F7B12C07C0C8
:101D9000BC2EB8018C2F0E94E3150197A9F38B2D5F
:101DA000DF91CF911F910F91FF90EF90DF90CF9037
:101DB000BF900895CF93DF93EC010E94980EBE016F
:101DC0000E94E315DF91CF9108951F93CF93DF9386
:101DD000EB019091F101992321F0CB010E94DA0EE1
:101DE00013C0882349F0CB010E94980E182F682F4A
:101DF000CE010E94410E04C0CB010E946C0E182F30
:101E0000BE01812F0E94E315DF91CF911F910895AC
:101E10001F93CF93DF93C091040216E080910502D7
:101E2000C81799F0D0E01C9FF0011D9FF00D112400
:101E3000EA5FFD4F40815181628173818481958188
:101E40000E94210D2196C770E9CFDF91CF911F919C
:101E50000895409136025091370260913802709196
:101E6000390280913A0290913B020C94210DEF923D
:101E7000FF920F931F93CF93DF9380913B02829544
:101E80008F7009F065C080913802882309F460C022
:101E900080910402F0900502109136020091370201
:101EA0006091390270913A0291E01F3F09F090E091
:101EB000C0910001D0910101292F96E0E92E8F15E4
:101EC00009F446C06115710521F00F3F21F030E0A3
:101ED00003C031E001C0322F90E030FD36C0E89EF3
:101EE000F001E99EF00D1124DF01AA5FBD4F1196AC
:101EF0003C911197301329C03C91311326C01296A2
:101F00003C911297311121C013964D915C91149719
:101F1000461B570B4C175D07C0F480913B028F7036
:101F2000806180933B02E55FFD4F80818F7080610F
:101F3000808386E392E00E949F0CDF91CF911F91F6
:101F40000F91FF90EF900C94080F01968770B7CF18
:101F5000DF91CF911F910F91FF90EF9008959F9285
:101F6000AF92BF92CF92DF92EF92FF920F931F93A7
:101F7000CF93DF93CDB7DEB761970FB6F894DEBF8E
:101F80000FBECDBF8C0185E0F801DE011D960190EA
:101F90000D928A95E1F7D8011296EC909091360255
:101FA000E09137022091390230913A022115310532
:101FB00031F0EF3F31F481E09F3F19F403C081E03D
:101FC00001C080E0B82FB1709B2E80FD47C1D801C1
:101FD0004C9111965C9111971396AD90BC9014970B
:101FE00086E3C82E82E0D82EF0903802B501621B3D
:101FF000730B2091000130910101FF2009F4D9C039
:1020000080913B026217730708F095C0282F207F4C
:1020100009F052C05E1313C0491311C0FE2CE11029
:102020000EC08F70806180933B020E94290FC60111
:102030000E949F0C80913B02F80185834DC1AB2823
:1020400031F05F3F31F481E04F3F19F403C081E08C
:1020500001C080E080FD03C081E08E2502C080E0E9
:1020600090E0F82FF170FF2E80FF1CC080910402D9
:102070002091050236E0821709F40BC190E0389FE9
:10208000F001399FF00D1124EA5FFD4F6181561375
:1020900006C06081461303C06281E61203C0019648
:1020A0008770E9CFFE2CEE2009F416C180913B0227
:1020B000816080933B0254C05E1306C0491304C084
:1020C000E11002C0F80199C0C8010E940A0D8823DE
:1020D00061F1EE2051F120913B02822F82958F70A9
:1020E00090E0029774F080913602909137029887C1
:1020F0008F831986BB86AA862C87CE0107960E94FD
:102100009F0C86E0F801A6E3B2E001900D928A955B
:10211000E1F70E94370F0E94290F0AC05E1711F1E4
:10212000C8010E940A0D81112CC0C8010E949F0C99
:10213000FF24F394D1C0282F207F81F77A2DB98A0C
:10214000A88A6E2D89890E94120D86E392E00E9472
:102150009F0C86E0D6011D928A95E9F70E94290F0F
:10216000F12CBAC04913DCCFE110DACFF801858336
:10217000C8010E949F0C86E0D6011D928A95E9F75E
:10218000ABC0EE2091F220913B02822F82958F709E
:1021900090E002970CF4B5CF80913602909137020F
:1021A0009A8389831B82BD82AC822E83CE010196E5
:1021B000A6CF6217730708F044C0FE2CEE2009F486
:1021C000B4CF5E1330C049132EC020913B0220FDD6
:1021D00021C0822F82958F70482F50E04115510504
:1021E000C9F0F80125834F30510541F08F5F982FDA
:1021F0009295907F822F8F70892B8583C8010E94D2
:102200009F0C86E0F801A6E3B2E001900D928A955A
:10221000E1F73CC086E0F801A6E3B2E001900D9240
:102220008A95E1F759C0C8010E940A0D811169CF52
:1022300080913B02816080933B02C8010E949F0C09
:102240004BC07A2DB98AA88A6E2D89890E94120DF9
:1022500086E0D6011D928A95E9F718C0EE2009F4B0
:1022600064CFC8010E940A0DF82E882309F45DCFBF
:1022700086E0F801A6E3B2E001900D928A95E1F7BD
:1022800086E392E00E940B090E94370F0E94290FFB
:1022900023C04D875E878D859E850E94DA0E292F8B
:1022A00022952F70223028F49F7039F0811105C0DB
:1022B0000BC0243028F49F7049F4805E883020F0F1
:1022C000C8010E949F0C9F2CF92C06C0D8011596BE
:1022D0009C91907F91F7F8CF8F2D61960FB6F8946F
:1022E000DEBF0FBECDBFDF91CF911F910F91FF9049
:1022F000EF90DF90CF90BF90AF909F9008951F9385
:10230000CF93DF93CDB7DEB72C970FB6F894DEBF2F
:102310000FBECDBF4F83588769877A878B879C878D
:10232000CE0107960E94AF0F8823D1F09F81888548
:102330002A853B85232B31F08F3F31F481E09F3F8D
:1023400019F403C081E001C080E080FD47C04F81E7
:10235000588569857A858B859C850E94210D3EC0B4
:1023600086E0FE013796DE01119601900D928A9566
:10237000E1F7FF81E8856A857B856115710531F09C
:10238000EF3F31F481E0FF3F19F403C081E001C069
:1023900080E080FD23C02091050230E0C901019654
:1023A000877099274091040250E084179507F1F156
:1023B000F983EA837D836C8396E0929FD001939F9B
:1023C000B00D1124AA5FBD4FFE01319601900D9210
:1023D0009A95E1F7809305020E94080F16E080911C
:1023E000040290910502891771F1189FC001112410
:1023F0008A5F9D4F0E94AF0F882329F1E09104026C
:102400001E9FF0011124EA5FFD4F408151816281DE
:102410007381848195810E94210D8091040290E056
:1024200001968770992780930402D9CF0E94EB0C04
:102430001092050210920402E6E3F2E086E0DF016A
:102440001D928A95E9F72C960FB6F894DEBF0FBE61
:10245000CDBFDF91CF911F91089580914402859562
:10246000859585950895809144028770089590918F
:102470004402977081E009F480E0089580914F0252
:10248000089590914F02892B80934F020895809573
:1024900090914F02892380934F02089510924F022A
:1024A000089590914E02892B80934E020895809555
:1024B00090914E02892380934E02089510924E020D
:1024C000089580914502089508950C9464120C9427
:1024D000651290918F0292FD08C090914502981765
:1024E00021F0809345020C94671208958091450273
:1024F000882329F01092450280E00C946712089519
:10250000CF93DF93E0910201F091030180914F029C
:102510008083E0910201F0910301908180914E024D
:10252000892B808380914502882381F0E09102010C
:10253000F09103019081892B808380910201909119
:1025400003010E94FE2381110E947612C0910201B4
:10255000D091030148E050E06CE372E0CE010E94AC
:10256000662D892B69F088E0FE01ACE3B2E00190B2
:102570000D928A95E1F7CE01DF91CF910C947B23E8
:10258000DF91CF9108950C94641290918F0292FD87
:1025900010C098E0899F90011124262B20934402BB
:1025A0000E94A30D809144028595859585950C9494
:1025B000C3120C94A30D1092440280E00C94C31239
:1025C000209144028095822380934402982F977033
:1025D00099F430E0482F082E000C550B24173507CE
:1025E00059F090918F0292FD07C08595859585954C
:1025F0000E94C40D0C94DB120895CF9390918F022A
:1026000092FB222720F92817F9F0C82F892FC0FB49
:1026100082F980938F0280918E0290918F020E94A6
:10262000591382E00E94E01280915B0280FF0CC08F
:102630001F92CF938EEF91E09F938F930E94840619
:102640000F900F900F900F90CF91089580918F026F
:1026500082FB882780F991E089270C94FD1281E0A4
:102660000C94FD1280E00C94FD1280E090E00E943A
:102670007B2D21E0893E9E4F09F020E0822F0895B6
:1026800082E090E00C94732D83E090E00C94732D25
:10269000CF9384E090E00E94732DC82F82E290E0F7
:1026A0000E94732D2C2F30E0A901582BCA01CF9125
:1026B0000895CF93C92F682F84E090E00E94812D68
:1026C0006C2F82E290E0CF910C94812DAB01BC0184
:1026D0008FE090E00C94932DAB01BC0183E190E07E
:1026E0000C94932D60E070E0CB010C946C1360E0CF
:1026F00070E0CB010E9466130C94721369EE7EEFBA
:1027000080E090E00E949F2D60E082E090E00E94D7
:10271000812D60E083E090E00E94812D1092000204
:1027200010920102109202021092030260E084E013
:1027300090E00E94812D60E082E290E00E94812D75
:1027400060E085E090E00E94812D60E086E090E00E
:102750000E94812D6FEF87E090E00E94812D40E084
:1027600050E0BA0188E090E00E94932D60E08DE097
:1027700090E00E94812D40E050E0BA0188E190E0B5
:102780000E94932D60E087E190E00E94812D40E05F
:1027900050E0BA018CE190E00E94932D60E070E07F
:1027A00080E290E00E949F2D40E050E0BA0188E175
:1027B00090E00E94932D0C9477130C947E13682F55
:1027C0008EE090E00C94812D0E94F22460935702D9
:1027D000709358028093590290935A026093530267
:1027E000709354028093550290935602089585B7D2
:1027F000806885BF85B7806885BF089581E00895AA
:102800000C94FE1308950C9402140C9402140C946E
:1028100005140C9402140C9409140C9402140E94D4
:10282000F7138AE297E20E9465230E940D140C942C
:102830000B140E9403140C9402140E94C0160E94F0
:102840007E080C94C91D0E94DD240E94D3170E94AB
:102850001D140E94961B0C9407148F929F92AF92A6
:10286000BF92CF92DF92EF92FF920F931F93CF937D
:10287000DF93CDB7DEB72A970FB6F894DEBF0FBE51
:10288000CDBF0E94E817982E81110E94E41380E5C5
:10289000A82E82E0B82E00E010E0802E802F0E944B
:1028A000E416D82EF501C1905F01C826B1F40F5F80
:1028B0001F4F0330110589F78FEF89838A831B82AD
:1028C0000E94E6248160782F9D838C8349815A8100
:1028D0006B818D810E94C1082FC080915B0281FDB8
:1028E0000E94EA16E12CFF24F3948C2D8F21F1F045
:1028F0000E940014882399F0EE828F82DF2081E00D
:1029000009F480E088870E94E6248160782F9A8706
:1029100089874E815F8168858A850E94C108F80198
:10292000E05BFD4F8081F826F08206C0E394FF0C47
:10293000F3E0EF12DACFBBCF81E0911001C080E06D
:102940002A960FB6F894DEBF0FBECDBFDF91CF91B0
:102950001F910F91FF90EF90DF90CF90BF90AF90BD
:102960009F908F9008950E942D140E94C81D0E9470
:10297000641A0C948F08CF93DF930E94E815EC0142
:10298000811521E5920708F045C0811530E59307D0
:1029900008F094C0883E910528F5803E910508F026
:1029A000F8C0883A910570F4853A910508F07CC02A
:1029B0008130910509F475C008F4E8C0049708F067
:1029C000E8C0E4C08F3B910508F0E0C0C85AD0E0F1
:1029D000CC0FDD1FC65BDE4F0990D881C02DCE0124
:1029E0009464D8C0811540E2940758F4811551E0F1
:1029F000950708F0CEC08D3E910508F4C7C09065DC
:102A0000C9C0C11580E4D80708F4C0C0DF70CE018A
:102A1000906AC0C0811525E59207A8F4811534E5B8
:102A2000930708F095C0811543E5940708F07BC033
:102A3000811552E5950708F061C0D82FCC27CE014B
:102A4000816F906AA7C0C11589E5D807A0F4C115A8
:102A500028E5D20708F082C0C11536E5D30708F093
:102A600095C08C2F0E947C168F7190E0D82FCC27B8
:102A7000CE0190628FC0C1154AE5D40708F474C036
:102A8000CE0190568115904208F080C08D2F8F7135
:102A90000E947C16DD27D0628F71AE01582BCA01CF
:102AA00079C081E090E076C0C55AD0E0C858DE4FCA
:102AB0008881C82FD0E0CE0190646CC074E09695F8
:102AC00087957A95E1F7282F23703C2F337081E0AA
:102AD00090E002C0880F991F3A95E2F79C68AC011C
:102AE000522B9A019C2F9F709695969550E2959F38
:102AF000E0011124C9018C2B9D2B4CC083709927B8
:102B000021E030E002C0220F331F8A95E2F79C2FAC
:102B10009695969580E2989FE0011124C22BD32BC5
:102B2000CE019C6837C08370992721E030E002C055
:102B3000220F331F8A95E2F79C2F9695969540E2D7
:102B4000949FE0011124C22BD32BCE019A6822C09E
:102B5000D82FCC27CE01846F906A1CC0DC2FCC27E5
:102B6000CE01806F906A16C08C2F8F700E947C16E9
:102B700094E0D695C7959A95E1F7CF70D0E0DC2F19
:102B8000CC27D0699E01282BC90104C080E090E0C9
:102B900001C0CE01DF91CF910895272F30E0F901D8
:102BA000EE0FFF1F2E0F3F1FF90199E0899FE00DE7
:102BB000F11D1124E60FF11DEE0FFF1FE95FFE4F1F
:102BC0008591949108950E94CD150E94BB1408959B
:102BD0008238910569F1B0F48133910509F46DC033
:102BE00048F48932910509F463C08A32910509F4E9
:102BF00069C008958533910509F455C0893391055D
:102C0000B9F00895833E910569F138F4803E91054D
:102C1000B1F0823E910509F10895863E9105A9F132
:102C2000873E9105B9F1843E910509F064C023C047
:102C300020918E0220FD4FC021FD4DC0089580914E
:102C40008E0280FD44C080918F0280FF44C080913D
:102C50008E0284FD42C083EE4DC080918E0282FFC1
:102C600038C0F5CF80918E0282FD33C080918F02F3
:102C700080FD31C0ECCF80918F0281FF32C0809106
:102C80008E0284FD2AC087EE35C080918E0283FFBC
:102C900026C0F5CF80918E0283FD21C080918F02E6
:102CA00081FD1FC0ECCF80918E0285FD1CC01DC030
:102CB00080918E0285FD19C016C080918E0286FD1E
:102CC00016C017C080918E0286FD13C010C089E324
:102CD00011C082EE0FC080EE0DC080E00BC086EE0A
:102CE00009C084EE07C089E205C085E303C08AE21B
:102CF00001C081E390E0089590918E0292FF0DC093
:102D0000282F2871283019F4877F846006C0282F67
:102D10002471243011F48B7F886093FF0DC0282F1D
:102D20002871283119F4877E846106C0282F247108
:102D3000243111F48B7E886120918F0220FF0DC019
:102D4000382F3871383019F4877F816006C0382FEA
:102D50003171313011F48E7F886021FF0DC0282F32
:102D60002871283119F4877E816106C0282F2171CE
:102D7000213111F48E7E886194FD877E0895089537
:102D80000E943513811102C00E94DD130E9440137E
:102D900080935B020E94481390938F0280938E026F
:102DA0000E94BF160E944413682F70E080E090E0FC
:102DB0000E94430D6091FC017091FD018091FE0124
:102DC0009091FF010C947B0DE82FF0E0ED56FD4F44
:102DD00080810895CF92DF92EF92FF920F931F931D
:102DE000CF93DF9382E292E00E94EB0583E9E82E25
:102DF00082E0F82EC0E0D0E09DE1C92E92E0D92E0D
:102E000005E112E0DF93CF93DF92CF920E94840618
:102E10008AE192E00E94EB05F70181917F010E9417
:102E200065081F928F931F930F930E94840683E17E
:102E300092E00E94EB0521968DB79EB708960FB6DB
:102E4000F8949EBF0FBE8DBFC330D105D9F6DF9178
:102E5000CF911F910F91FF90EF90DF90CF90089549
:102E600080EA8A95F1F7089500C008950C94301710
:102E700008950C9438170C9439170C9438170C9447
:102E80003D17F894E82FE295EF70F0E031A1282F7C
:102E90002F7081E090E001C0880F2A95EAF7982F03
:102EA0009095932391A392A1892B82A3789408955E
:102EB00081E90E94411780E90E94411784E90E943C
:102EC000411786EC0E94411787E90E94411786E668
:102ED0000C944117EF92FF920F931F93CF93DF93C0
:102EE000C62FD0E0C558DE4F28812F3F09F454C0CB
:102EF000042F162F7C01F894E22FE295EF70F0E09A
:102F000081A1422F4F7021E030E001C0220F4A958D
:102F1000EAF7822B81A382A12095282322A378940B
:102F20000E9434176EE771E0F701A7014D5F5F4F14
:102F3000F12C302F3095DB012D91BD012F3FB1F0E9
:102F4000822F82958F7090E0DC0190968C9190E0BA
:102F50002F7002C0959587952A95E2F780FD06C0EF
:102F60008081802B8083FF24F39403C0808183239E
:102F700080833196E417F507F1F688818F3F11F0D1
:102F80000E9441176F2D812FDF91CF911F910F91DB
:102F9000FF90EF900C943617DF91CF911F910F9116
:102FA000FF90EF9008950E94581783E0E3E9F2E064
:102FB000DF01982F1D929A95E9F7E0E9F2E0DF0131
:102FC0001D928A95E9F783E00E942A180C94F60670
:102FD0000F931F93CF93DF9300D01F92CDB7DEB72F
:102FE00019821A821B8210E001E0402F612FCE016E
:102FF00001960E946A171F5F000F1330B1F743E07C
:1030000050E0BE016F5F7F4F80E992E00E94662D25
:1030100011E0009709F410E0892B49F089819A8129
:10302000AB818093900290939102A0939202212F02
:1030300043E063E972E080E992E00E942B180E946D
:10304000F806812F0F900F900F90DF91CF911F9175
:103050000F9108950895FF920F931F93CF93DF93DD
:103060008C01F62ED72FC42F222349F081E08093C4
:103070005E020E94E62490935D0280935C02809140
:103080005E028823C1F080915C0290915D020E94F3
:10309000FE24059780F0EF2DFD2FD8014C2F50E036
:1030A000CD01801B910B841795071CF48D918193A2
:1030B000F7CF10925E02DF91CF911F910F91FF9099
:1030C00008950E94A6270E9423140C94B2270E9400
:1030D000B6270E94B3140C94D4270E9484240E9423
:1030E0008D270E940F140E9461180E9467180E9489
:1030F0001914FBCF8091650280FF06C06091090121
:1031000070E0660F771F26C081FF04C0609109013F
:1031100084E005C082FF07C06091090188E0689FD4
:10312000B001112417C0909164029923D1F06091ED
:103130000801961788F72091090188E0289F9001DF
:103140001124929FA001939F500D112470E0CA0199
:103150000E94102D6038710540F46115710519F455
:1031600006C068E070E0862F08958FE7089581E03B
:1031700008958091650280FF08C06091050170E0AC
:10318000759567957595679521C081FF06C060911B
:10319000050170E07595679519C082FF04C06091C4
:1031A000050170E010C090916302992399F060913D
:1031B00004019617A0F780910501899FC001112491
:1031C00070E00E94102D6038710540F461157105A2
:1031D00019F406C061E070E0862F08958FE7089526
:1031E00081E008958D3E21F40E947A18819504C0F3
:1031F0008E3E29F40E947A188093690208958F3ECA
:1032000021F40E947A18819504C0803F29F40E941D
:103210007A18809368020895893F19F40E94B918BA
:1032200005C08A3F31F40E94B918819580936A02E3
:1032300008958B3F21F40E94B918819504C08C3FFA
:1032400029F40E94B91880936B0208959FE0980FAB
:10325000983078F421E030E0A90102C0440F551FF6
:103260009A95E2F7CA0190916702892B80936702D1
:1032700008958D3F21F48091650281600BC08E3FDF
:1032800021F480916502826005C08F3F29F480910E
:10329000650284608093650208958D3E39F49091B3
:1032A000690297FF35C01092690259C08E3E29F419
:1032B000909169021916BCF32BC0909168028F3E61
:1032C00029F497FF25C01092680249C0803F19F485
:1032D0001916CCF31DC090916A02893F29F4191682
:1032E000BCF410926A023BC08A3F19F497FF10C0E9
:1032F000F8CF8B3F39F490916B0297FF09C0109281
:103300006B022DC08C3F21F490916B021916BCF317
:103310009FE0980F983080F421E030E0A90102C0CE
:10332000440F551F9A95E2F7CA0180959091670264
:1033300089238093670213C08D3F21F48091650239
:103340008E7F0BC08E3F21F4809165028D7F05C07A
:103350008F3F29F4809165028B7F80936502809175
:103360006802811106C080916902811102C0109229
:10337000640280916A02811106C080916B02811102
:1033800002C010926302089580915B0283FF7EC0A9
:1033900088E592E00E94EB05809167021F928F936F
:1033A00083E592E09F938F930E94840681E592E0EB
:1033B0000E94EB0580916802282F082E000C330B29
:1033C0003F938F938EE492E09F938F930E948406A5
:1033D0008CE492E00E94EB0580916902282F082E70
:1033E000000C330B3F938F9389E492E09F938F936C
:1033F0000E94840687E492E00E94EB0580916A02B5
:10340000282F082E000C330B3F938F9384E492E017
:103410009F938F930E94840682E492E00E94EB05C2
:1034200080916B02282F082E000C330B3F938F9353
:103430008FE392E09F938F930E9484068CE392E047
:103440000E94EB05809164021F928F9389E392E0C2
:103450009F938F930E94840687E392E00E94EB057E
:10346000809165021F928F9384E392E09F938F93E4
:103470000E94840681E392E00E94EB058DB79EB71F
:103480004C960FB6F8949EBF0FBE8DBF0E94E624E7
:1034900020916802211104C020916902222321F0A9
:1034A000909362028093610220916A02211104C00C
:1034B00020916B02222321F09093600280935F029F
:1034C00086E692E00C94C423EF92FF920F931F9331
:1034D000CF93DF9300D000D000D0CDB7DEB786E029
:1034E000E6E6F2E0DE01119601900D928A95E1F791
:1034F000E0906802F090690200916A0210916B02FC
:10350000109268021092690210926A0210926B0285
:10351000E11003C0FF2009F45DC080916102909129
:1035200062020E94FE24AC0190916402992339F05A
:1035300020910A0130E02417350758F04BC0209144
:103540000B018AE0289F900111242417350718F0F9
:1035500041C09F3F19F09F5F90936402EE2061F09D
:103560000E947A181E1414F09FEF01C091E0989FFA
:10357000902D112490936802FF2061F00E947A1828
:103580001F1414F09FEF01C091E0989F902D11241B
:1035900090936902309168023323E1F0209169022F
:1035A0002223C1F045EB3403C0011124992319F003
:1035B0009093680203C081E08093680235EB230397
:1035C000C0011124992319F09093690203C081E08E
:1035D00080936902011103C0112309F45DC0809139
:1035E0005F02909160020E94FE24AC019091630200
:1035F000992339F02091060130E02417350758F05F
:103600004BC0209107018AE0289F900111242417C4
:10361000350718F041C09F3F19F09F5F90936302F8
:10362000002361F00E94B918101614F09FEF01C03A
:1036300091E0989F902D112490936A02112361F0DC
:103640000E94B918111614F09FEF01C091E0989FE5
:10365000902D112490936B0230916A023323E1F094
:1036600020916B022223C1F045EB3403C0011124E9
:10367000992319F090936A0203C081E080936A0253
:1036800035EB2303C0011124992319F090936B02A9
:1036900003C081E080936B028091680281110BC0AE
:1036A00080916902811107C080916A02811103C073
:1036B00080916B0281110E94C419EB82FC820D8300
:1036C0001E8386E0FE013196A6E6B2E001900D92DF
:1036D0008A95E1F726960FB6F894DEBF0FBECDBFF0
:1036E000DF91CF911F910F91FF90EF900895E6E643
:1036F000F2E086E0DF011D928A95E9F710926402FC
:103700001092630210926502089586E090E00C9496
:10371000732D682F86E090E00C94812D80919602A5
:1037200084708165809396020C94891B0E943513E6
:10373000811104C00E94DD130E948E1B0E94851B14
:1037400080939602282F26952695269530E02B30DB
:10375000310524F0877080658093960280919602EF
:1037600080FF04C086958695869501C080E00C9404
:10377000131D20919602822F869586958695482F57
:1037800050E04A30510554F48F5F982F990F990FEC
:10379000990F822F8770892B8093960280919602D1
:1037A0008160809396020E94891B80915B0280FF5A
:1037B00011C0809196028695869586951F928F936B
:1037C00082EE92E09F938F930E9484060F900F9059
:1037D0000F900F90809196028695869586950C9411
:1037E000131D80919602982F969596959695A1F027
:1037F000915E990F990F990F8770892B809396028C
:10380000887F91E009F490E08091960290FB80F926
:10381000809396020E94891B80915B0280FF11C0F9
:10382000809196028695869586951F928F938AEC55
:1038300092E09F938F930E9484060F900F900F90B9
:103840000F90809196028695869586950C94131D0F
:103850008091960280FD1FC0816080939602813026
:1038600019F489E080939602809196020E94891B48
:1038700080915B0280FF08C082EA92E09F938F9361
:103880000E9484060F900F908091960286958695EF
:1038900086950C94131D08958091960280FF14C0A4
:1038A0008E7F809396020E94891B80915B0280FF2D
:1038B00008C08FE892E09F938F930E9484060F9038
:1038C0000F9080E00C94131D0895CF93C091960241
:1038D000C17080915B0280FF0CC01F92CF9384EB7C
:1038E00092E09F938F930E9484060F900F900F9009
:1038F0000F90CC2319F0CF910C944C1CCF910C94C9
:10390000281C90919602892F8695869586958F5FC3
:103910008F7197708B3038F4880F880F880F892B40
:103920008093960202C09093960280919602887FBF
:1039300091E009F490E08091960290FB80F98093E9
:1039400096020E94891B80915B0280FF11C08091CA
:1039500096028695869586951F928F938BE792E0C7
:103960009F938F930E9484060F900F900F900F905B
:10397000809196028695869586950C94131D8B30C2
:1039800008F08AE0909196029770282F220F220F5C
:10399000220F922B90939602987F21E009F420E069
:1039A0009091960220FB90F9909396020C94131D2F
:1039B0000E94BF1C809196020C94891B9C01FB0104
:1039C0008281882349F12E3BFCE53F07C9F040F492
:1039D0002C3BECE53E0769F02D3B3C4561F008953A
:1039E000203C9CE5390791F070F0213C3C4589F082
:1039F00008958AE001C080E00E94D81C80E008950C
:103A00000E94F11BFBCF0E94B91BF8CF0E94651CDE
:103A1000F5CF0E94811CF2CF81E00895259A2D9860
:103A200008952D9808958F929F92AF92BF92CF9252
:103A3000DF92EF92FF920F931F93CF93DF93C82FE4
:103A40008B3050F4811109C0809180008F77809372
:103A500080000E94111D06C0CAE08091800080682D
:103A600080938000A0918600B09187002C2F30E0D9
:103A70000E944C2D2AE030E040E050E00E94242DCE
:103A80000027122F232F342F012F122F232F3327FC
:103A900080918600909187006CE070E00E94FC2C81
:103AA0006017710730F0C80169E070E00E94FC2CDB
:103AB0005EC08091860090918700E0908600F09033
:103AC0008700E0918600F0918700C6E0D0E0BE015B
:103AD0000E94FC2C060F171F211D311D48015901A2
:103AE00085E0880C991CAA1CBB1C8A95D1F7C701DC
:103AF000BE010E94FC2C6F01E12CF12CA701960164
:103B0000260F371F411D511DC501B4010E94242DF0
:103B100069017A01E0918600F0918700CA01B9013C
:103B20000E94E02C9B01AC01DF010E945B2D9B01F8
:103B3000AC01C701B6010E94E02CDC01CB012FE0F3
:103B4000B695A795979587952A95D1F70091860008
:103B50001091870020E030E0081719072A073B077B
:103B600028F46091860070918700CB01BC017093AE
:103B7000890060938800DF91CF911F910F91FF9092
:103B8000EF90DF90CF90BF90AF909F908F9008956F
:103B900008950E940E1D82E88093800089E1809341
:103BA00081008FEF9FEF90938700809386000C94A5
:103BB000961BCF93DF93EC01FB018281882309F4EC
:103BC0003CC1C430FDE5DF0760F4CB3F9CE5D9077D
:103BD00088F49E0122503C452431310508F02EC165
:103BE00009C0C236EDE5DE0729F0C63AFDE5DF077C
:103BF00009F024C10E94481390938F0280938E0293
:103C0000C1318CE5D80709F4C6C008F042C0C930FC
:103C1000ECE5DE0709F49BC000F5C5308CE5D8075C
:103C200009F485C078F4C330ECE5DE0709F478C008
:103C300008F07AC0C230DC4509F0F5C080918E02F0
:103C40008160EFC0C7309CE5D90709F478C008F05F
:103C50007AC080918E028061E4C0CD30FCE5DF0740
:103C600009F487C058F4CB309CE5D90709F479C032
:103C700008F07BC080918E0288606FC0CF30FCE579
:103C8000DF0709F480C008F082C080918E02877F30
:103C9000C8C0CE3F9CE5D90709F471C000F5C53115
:103CA000FCE5DF0709F485C068F4C3319CE5D9075A
:103CB00009F475C008F095C00E94EB0C80918E024B
:103CC0008F77AFC0CC3FFCE5DF07A9F108F054C007
:103CD000CB3FDC4509F0A7C080918F0240C0C230C5
:103CE000EDE5DE0709F489C058F4C1158DE5D80764
:103CF00009F45AC008F069C080918F0282602FC019
:103D0000C236EDE5DE0709F47CC0C63AFDE5DF0703
:103D100009F481C0C330DD4509F085C080E06EC084
:103D200080918E0282607DC080918E0216C080914B
:103D30008E02886076C080918F0282604FC0809131
:103D40008E0280626EC080918E0280646AC00E9482
:103D5000EB0C80918E02806864C0846062C08160D8
:103D60003DC080918E028E7F5CC080918E028D7FDF
:103D700058C080918E0216C080918F0218C0809129
:103D80008F028D7F2BC080918E028F7E4AC08091E2
:103D90008E028F7D46C080918E028F7B42C08091C3
:103DA0008E02877F8B7F3DC080918F028D7F8E7FBB
:103DB00015C080918E0282FB222720F991E0922784
:103DC00090FB82F990FB83F92CC080918F02982F91
:103DD000909591708E7F892B90FB81F980938F0253
:103DE00022C00E94EB0C80918E0287FB222720F9D3
:103DF00091E0922790FB87F914C081E00E94DF13C5
:103E000012C080918E0284FB222720F991E0922734
:103E100090FB84F906C080918E02982F909590FBBC
:103E200080F980938E0280918E0290918F020E9481
:103E300059130E94EB0C80E001C081E0DF91CF912B
:103E40000895809104011F928F93809105011F9224
:103E50008F93809108011F928F93809109011F9287
:103E60008F9380910A011F928F9380910B011F9273
:103E70008F938AEF92E09F938F930E9484068DB771
:103E80009EB70E960FB6F8949EBF0FBE8DBF0895D5
:103E9000883220F58E3108F068C08B3091F1C0F483
:103EA000873009F0BEC081E080930B0184E18093EC
:103EB0000A018AE0809309018EE18093080188E07D
:103EC0008093050188E2809304018CE594E0C6C0EC
:103ED000833109F443C0843169F1A3C08F3409F4FC
:103EE0009EC028F4893231F1883359F09AC0813567
:103EF00031F008F4D4C0823509F4A7C092C08FEF26
:103F0000A5C08EE794E00E94EB050E94211F1F923E
:103F100081E08F931F9288E08F9387E793E09F93D0
:103F20008F930E9484060F900F900F900F900F9028
:103F30000F9096C08BE794E00E94EB058091700291
:103F4000882309F4AAC01092700210926F02109296
:103F50006E0210926D0210926C02B1C08DE694E078
:103F60000E94EB050E94211F7BC08D51809370023F
:103F7000833031F170F48130D1F0823009F03FC0EC
:103F80008AE091E090936F0280936E028EE891E058
:103F90001FC0853059F108F1863089F584E091E041
:103FA00090936F0280936E0289EC91E011C08BE0D8
:103FB00091E090936F0280936E0285E891E008C0D3
:103FC00089E091E090936F0280936E028AE991E01C
:103FD00090936D0280936C0218C088E091E09093FA
:103FE0006F0280936E0287EA91E0F2CF85E091E064
:103FF00090936F0280936E0286EB91E0E9CF10926E
:1040000070028AE694E00E94EB058091700288239A
:1040100009F455C01F928F9386E694E00DC08AE0A4
:1040200015C089E594E01AC097FF47C010828081CF
:104030001F928F9383E594E09F938F930E94840651
:104040000F900F900F900F900BC081E0E0916E02E7
:10405000F0916F02309729F580E594E00E94EB051E
:1040600020917002222359F180916C0290916D028F
:10407000009711F481E891E09F938F931F922F9303
:1040800087E494E09F938F930E9484060F900F9093
:104090000F900F900F900F9016C080E0089586EF5C
:1040A000D5CF2081082E000C990B820F911D8F3FD8
:1040B000910509F00CF4B8CF8FEF8083B8CF83E47B
:1040C00094E00E94EB0581E00895CF93C82F1F92E2
:1040D0008F9384E994E09F938F930E94840681E0FC
:1040E00090E0A0E0B0E0BC01CD0104C0660F771FF6
:1040F000881F991FCA95D2F70E94430D0F900F9009
:104100000F900F90CF910C94EB0CEF92FF920F93C6
:104110001F93CF93DF938B3109F409C108F0AAC034
:104120008B3009F4CDC008F094C0863009F4CBC0C0
:1041300020F4853009F4D9C06AC1873009F4DCC0A5
:10414000883009F064C10E9444131F928F9389EE56
:1041500098E09F938F930E9484060E94401383FBF4
:10416000992790F91F929F9382FB992790F91F92AC
:104170009F9381FB992790F91F929F93982F91709D
:104180001F929F931F928F9380EA98E09F938F9343
:104190000E9484060E94481387FB222720F91F9261
:1041A0002F9386FB222720F91F922F9385FB22272E
:1041B00020F91F922F9384FB222720F91F922F931F
:1041C00083FB222720F91F922F9382FB222720F9BD
:1041D0001F922F9391FB222720F91F922F93292FB3
:1041E00021701F922F9381FB222720F91F922F937A
:1041F000282F21701F922F939F938F938BEB97E023
:104200009F938F930E9484068DB79EB788960FB6B2
:10421000F8949EBF0FBE8DBF0E94851B982F969568
:10422000969596951F929F93982F91701F929F93AA
:104230001F928F9388E897E09F938F930E94840644
:104240008DB79EB708960FB6F8949EBF0FBE8DBF70
:1042500035C0803109F495C020F48E3009F47BC05C
:10426000D6C0863109F4A8C0893109F0D0C084E0F5
:1042700095E084C08A32E1F060F4873209F4C3C06B
:1042800028F48E3108F4C3C08D51BEC0893269F163
:10429000BEC0833448F48A3308F0B3C0853309F4D0
:1042A000B2C0883369F0B3C0833409F4ACC0AFC086
:1042B00084E999E00E94EB050E94DD13C1E0ACC0E7
:1042C00085EE95E05BC080915B02817F8E7F80935D
:1042D0005B028EEB95E00E94EB0580E999E00E947D
:1042E000EB0581E080937102E9CF84E799E00E94B9
:1042F000EB050E94FB06E2CF80915B02C82FC095C0
:10430000C170C0FB80F980935B02CC2329F088E662
:1043100099E00E94EB0580C08BE599E00E94EB05D7
:1043200080915B02897F877F80935B02C7CF9091EA
:104330005B0291FBCC27C0F981E0C827892FC0FB25
:1043400081F980935B02CC2319F08EE499E029C0B7
:1043500080E499E013C090915B0292FBCC27C0F9F6
:1043600081E0C827892FC0FB82F980935B02CC23B0
:1043700019F081E399E015C081E299E00E94EB0514
:104380009DCF90915B0293FBCC27C0F981E0C827B9
:10439000892FC0FB83F980935B02CC2351F085E128
:1043A00099E00E94EB0580915B02816080935B0243
:1043B00033C088E099E0E2CF0E94F224162F072F45
:1043C000F82EE92ED0918D02C09118010E946F2322
:1043D000EF92FF920F931F931F92DF931F92CF9341
:1043E0001F928F9389E994E09F938F930E94840694
:1043F0008DB79EB70C960FB6F8949EBF0FBE8DBFBB
:104400005DCF895301C080E00E94652057CF86E0D0
:1044100099E00E94EB05C0E08C2FDF91CF911F91B6
:104420000F91FF90EF90089580E008950C9414226E
:10443000CF93C82F80917102813071F040F08230AB
:1044400009F045C08C2F0E94481F81E046C00E94A1
:104450003E128232F1F504C00E943E12823261F4B3
:104460008C2F0E941622811104C08C2F0E9485205F
:104470002CC081E090E029C08C2F0E941422811171
:1044800023C0C431C9F058F4CB3069F0C031B9F45D
:1044900082E08093710288E30E94481F15C0C932F0
:1044A00059F0C83361F48EEB95E00E94EB0580E98A
:1044B00094E00E94EB0508C0109271020CC08EE8D7
:1044C00094E00E94EB0507C081E0817006C0109265
:1044D000710280E002C080E0F8CFCF910895CF93C1
:1044E000DF9386319C4541F5EB010E943E12982FE7
:1044F0008A812091020130910301882379F09A7A10
:1045000081E009F480E080937202911102C069E2B7
:1045100001C065E3C9010E9440240AC08091720273
:10452000811102C069E201C065E3C9010E94422411
:104530000E94801280E001C081E0DF91CF91089558
:104540000F931F93CF93DF93C42FD22FFC0182814F
:104550008823C9F0409375020E94E6249093740268
:104560008093730280E28C0F883008F057C0C770C8
:1045700081E001C0880FCA95EAF7DF91CF911F91C2
:104580000F910C94480A80917502481330C08091B5
:104590007302909174020E94FE24883C910538F5C4
:1045A00010E21D0FCD17B9F080E28C0F883040F477
:1045B000C77081E001C0880FCA95EAF70E944F0AD0
:1045C000183028F581E09D2F977001C0880F9A95CB
:1045D000EAF70E94480A802F0E943F0A1830F0F440
:1045E000D77081E001C0880FDA95EAF70AC080E24F
:1045F0008C0F883098F4C77081E001C0880FCA958D
:10460000EAF7DF91CF911F910F910C944F0A802F01
:10461000DF91CF911F910F910C943F0ADF91CF91C1
:104620001F910F9108950F939C01CB01243F4CE5FE
:10463000340731F188F4293DFCE53F07D9F02A3DE4
:104640004CE5340779F1283D3C45A9F506E221EE19
:1046500041EE68ED7CE52BC0263FFCE53F07E1F02D
:10466000A8F0273F3C4539F507E225EE46EE67EF17
:104670007CE51DC007E225EE45EE69ED7CE517C03F
:1046800006E221EE40EE64EF7CE511C007E225EE84
:1046900044EE65EF7CE50BC006E221EE42EE66EFEC
:1046A0007CE505C008E221E045EE6AED7CE50E946C
:1046B000A02280E008C0FC018281882319F01092BA
:1046C000750201C081E00F9108959093EF018093EE
:1046D000EE01089590937B0280937A020895E09111
:1046E0007A02F0917B02309721F00190F081E02D69
:1046F000099480E00895EF92FF920F931F93CF9358
:10470000DF93E0917A02F0917B023097B1F18C0156
:104710000280F381E02D099580915B0282FF2DC01C
:1047200080FF04C08DEA99E00E94EB05E80118E0E3
:1047300087EAE82E89E0F82E80915B0280FF0BC0AB
:1047400088811F928F93FF92EF920E9484060F90B0
:104750000F900F900F90115021961111EDCF809175
:104760005B0280FF0AC085EA99E0DF91CF911F913B
:104770000F91FF90EF900C94EB05DF91CF911F917B
:104780000F91FF90EF900895E0917A02F0917B02F3
:10479000309739F022E0DC012C930480F581E02D84
:1047A00009940895209178023091790228173907E9
:1047B00071F09093790280937802E0917A02F091FF
:1047C0007B02309721F00680F781E02D099408954F
:1047D00020917602309177022817390771F0909373
:1047E000770280937602E0917A02F0917B02309713
:1047F00021F00084F185E02D09940895FC013296A2
:1048000097E080E0915029F021912223D9F38F5F26
:10481000F9CF0895662349F0FC013296089621915C
:10482000621729F0E817F907D1F780E0089581E0D1
:1048300008959C01FC0132969FEF80E0419146175C
:1048400089F09F3F19F4411101C0982F8F5F863086
:10485000A9F79F3F39F0F901E90FF11D97FDFA958E
:104860006283089508959C012A5F3F4FFC014281B5
:10487000461301C01282019682179307B9F7089573
:104880000C9419240C943324029626E0FC01119216
:104890002A95E9F7089508950C944B2483E08093BA
:1048A0007C020C944C24811102C081E001C082E0A2
:1048B00080937C020C944C240C94532481E08093CC
:1048C0007C020C944C240C945E2408950C94652472
:1048D0000C9466240C9465240C9465240C94652433
:1048E000CF930E946C240E94E8170E946A24C0E0C3
:1048F0008C2F0E94E416811104C0CF5FC330C1F732
:1049000001C081E0CF91089508951F920F920FB6D4
:104910000F9211248F939F93AF93BF9380917D0249
:10492000811113C08091970290919802A0919902F1
:10493000B0919A024196A11DB11D80939702909368
:104940009802A0939902B0939A02BF91AF919F9160
:104950008F910F900FBE0F901F90189580919F021E
:10496000843031F10E94820710927D0220E488E1B8
:1049700090E00FB6F894A895809360000FBE209346
:10498000600083B7817F846083BF83B7816083BF0A
:104990007894889583B78E7F83BF0FB6F894A895D7
:1049A00080916000886180936000109260000FBE6B
:1049B00008950E94EB0C0C94890782E084BD93E07B
:1049C00095BD9AEF97BD80936E0008952FB7F89428
:1049D0008091970290919802A0919902B0919A02C9
:1049E0002FBF08952FB7F8946091970270919802A5
:1049F0008091990290919A022FBF08959C014FB720
:104A0000F8948091970290919802A0919902B091A8
:104A10009A024FBF821B930B089578941F920F92B6
:104A20000FB60F9211248F939F93AF93BF938091F2
:104A3000970290919802A0919902B0919A020196E2
:104A4000A11DB11D8093970290939802A0939902A3
:104A5000B0939A02BF91AF919F918F910F900FBE2B
:104A60000F901F90189581E08093E00080E2809382
:104A7000D8001092C9008FE19EE40197F1F700C0C1
:104A8000000087E090EBDC018093A8029093A902DC
:104A9000A093AA02B093AB029CE088E10FB6F89411
:104AA000A895809360000FBE90936000FFCF809127
:104AB0008C020895089522E02093E9002FEF3091B1
:104AC000E800215035FD06C035ED3A95F1F70000BC
:104AD0002111F5CF2091E80025FF0BC040E050E008
:104AE00066E070E00E9443288091E8008E77809312
:104AF000E8000895CF93DF9321E02093E9002FEFA2
:104B00003091E800215035FD06C035ED3A95F1F7BA
:104B100000002111F5CF2091E80025FF14C0EC0121
:104B200040E050E068E070E00E9443288091E80097
:104B30008E778093E80088E0FE01A4E8B2E001905F
:104B40000D928A95E1F7DF91CF91089580938002CD
:104B5000709382026093810280919F02843001F5FC
:104B600082E08093E9008FEF9091E800815095FDFD
:104B700006C095ED9A95F1F700008111F5CF80916F
:104B8000E80085FF0DC040E050E063E070E080E8A1
:104B900092E00E9443288091E8008E778093E8009D
:104BA0000895BC0184E00C94A625BC0183E00C941C
:104BB000A62583ED99E00E94EB0580919E0281116C
:104BC00009C00E94D4290E94312A8091E2008460A9
:104BD0008093E20008958FEC99E00E94EB0510921B
:104BE0009E0208958BEC99E00E94EB050C946324DF
:104BF00087EC99E00E94EB0560919B0281E06111D6
:104C000001C080E00C944E2483EC99E00E94EB05F7
:104C100090919F0281E0943009F080E060919B02C6
:104C20000C94532420917F022F5F822F62E30E9415
:104C3000F02C992319F020937F02089510927F029F
:104C400080918302882371F180919F02843041F525
:104C50008091E9008F702091EC00922F917020FDDF
:104C600090E8892B93E09093E9009091EB0090FFFE
:104C700014C09091EE0097FF10C09091E80095FF4E
:104C800003C01092F100F9CF9091E80090FF05C0A9
:104C90009091E8009E779093E8008F708093E900F0
:104CA00010928302089542E061EC81E00E944D2958
:104CB00042E261EC82E00E944D2942E261EC83E035
:104CC0000E944D2990919F0281E0943009F080E08C
:104CD00060919B020C945C248091A102833009F4C2
:104CE00061C030F4813071F0823009F49AC00895C7
:104CF0008A3009F486C08B3009F46CC0893009F021
:104D0000A8C020C08091A002813A09F0A2C0809181
:104D1000E800877F8093E8008091A4029091A5022B
:104D2000892B21F468E084E892E003C060E080E031
:104D300090E070E00E948E288091E8008B7780934D
:104D4000E80008958091A002813209F082C080912C
:104D5000A4029091A502029708F07BC08091E80020
:104D6000877F8093E8008091E80082FD05C08091F4
:104D70009F028111F8CF6DC02091F3008091F20065
:104D800090E0922B029731F48091F100813011F084
:104D9000863021F48091F10080938C028091E800AC
:104DA0008B7753C08091A002813A09F052C0809164
:104DB000A4029091A502892B09F04BC08091E800D4
:104DC000877F8093E8008091E80080FFFCCF80918E
:104DD000180136C08091A0028132D9F58091A402D9
:104DE0009091A502892BA9F58091E800877F809397
:104DF000E8000E9482298091A202809318010C94FD
:104E0000EB0C8091A002813221F58091E800877F30
:104E10008093E8000E9482298091A30280938D02F2
:104E200008958091A002813AA1F48091E800877FE3
:104E30008093E8008091E80080FFFCCF80918D0294
:104E40008093F1008091E8008E778093E8000C94C5
:104E5000822908959FB7F894109283029FBF909182
:104E60009F02943009F057C09091E9009F703091F3
:104E7000EC00232F217030FD20E8922B23E02093BB
:104E8000E9002091EB0020FF43C02091EE0027FFB6
:104E90003FC020917E02222321F02091E80025FFCF
:104EA00037C010927E0226E03091E80035FD15C033
:104EB00030919F02343061F53091EB0035FD28C010
:104EC000215021F481E080937E0222C0EFE9FFE0CF
:104ED0003197F1F700C00000E7CF8093F100809197
:104EE000E80085FD0AC08091E80080FFFCCF80913A
:104EF000E8008E778093E80006C08FB7F89421E031
:104F0000209383028FBF9F709093E90080E0089503
:104F10009F709093E9008FEF089584B7877F84BFD7
:104F20000FB6F894A8958091600088618093600026
:104F3000109260000FBE90E080E80FB6F894809366
:104F40006100909361000FBE0C945E240E94D429EE
:104F50000E94312AE2EEF0E08081846080837894C0
:104F60000C94C52C8CE091E00C946A2380919F02F4
:104F70008530C9F48FEB99E00E94EB0580919F0288
:104F8000853079F40E94AE2480919D028823B1F38C
:104F90000E947024882391F30E942D280E94EB0C1C
:104FA000EDCF0C94D924089508950C94D727292F78
:104FB000332723303105C9F060F42130310581F009
:104FC0002230310509F041C08BE590E02FEF39E048
:104FD00040C021323105E1F02232310531F135C0D6
:104FE00082E190E02AE53AE034C0992781309105CA
:104FF00049F028F0029749F5E7EDF9E005C0EBEF3D
:10500000F9E002C0E7EEF9E0849190E09F0121C051
:1050100063307105D0F4660F771FFB01E951FE4F35
:105020002081318189E090E014C06330710568F41B
:10503000FB01EE0FFF1FEF51FE4F20813181FB017D
:10504000E252FE4F808190E004C080E090E020E0DA
:1050500030E0FA0131832083089580E189BD82E147
:1050600089BD09B400FEFDCF8091D8008F7D80936B
:10507000D8008091E00082608093E0008091E000A1
:1050800081FDFCCF0895CF92DF92EF92FF920F93B4
:105090001F93CF93DF93EC018B017A010E94A1292A
:1050A000811133C0E114F10439F0F701808191815D
:1050B000081B190BC80FD91FC12CD12C01151105C4
:1050C00019F18091E80085FD16C08091E8008E7787
:1050D0008093E800E114F10449F0F70180819181A7
:1050E000C80ED91ED182C08285E00FC00E94A129BE
:1050F000882321F30AC089918093F100015011099E
:10510000FFEFCF1ADF0ADACF80E0DF91CF911F9156
:105110000F91FF90EF90DF90CF9008952091A6021D
:105120003091A7022617370748F06115710539F449
:105130002091E8002E772093E80001C0B901FC011E
:1051400020E06115710579F180919F028823F1F1CA
:105150008530F1F18091E80083FD3CC08091E8004A
:1051600082FD2EC08091E80080FFEBCF2091F300FC
:105170008091F20090E0922B6115710551F088301A
:10518000910538F421912093F10061507109019645
:10519000F3CF21E0089709F020E08091E8008E77B6
:1051A0008093E800CECF2111CFCF0AC080919F021B
:1051B000882361F0853061F08091E80083FD0AC0AA
:1051C0008091E80082FFF2CF80E0089582E00895A8
:1051D00083E0089581E008952091A6023091A7020E
:1051E0002617370748F06115710539F42091E8005A
:1051F0002E772093E80001C0B901FC0120E0611581
:10520000710591F180919F02882309F440C0853097
:1052100009F43FC08091E80083FD3DC08091E80023
:1052200082FD2FC08091E80080FFE9CF2091F3003C
:105230008091F20090E0922B6115710559F0883051
:10524000910540F424912093F10031966150710949
:105250000196F2CF21E0089709F020E08091E80064
:105260008E778093E800CBCF2111CCCF0AC08091FC
:105270009F02882361F0853061F08091E80083FD12
:105280000AC08091E80082FFF2CF80E0089582E0BA
:10529000089583E0089581E00895982F973068F588
:1052A0009093E900981739F07091EC002091ED008F
:1052B0005091F00003C0242F762F50E021FD02C052
:1052C0009F5FECCF3091EB003E7F3093EB0030914D
:1052D000ED003D7F3093ED003091EB003160309375
:1052E000EB007093EC002093ED005093F0002091C0
:1052F000EE0027FDE5CF80E008958F708093E900F0
:1053000081E008958091A00287FF11C08091E8009C
:1053100082FD05C080919F028111F8CF11C080915C
:10532000E8008B770BC080919F02882349F0809121
:10533000E80080FFF8CF8091E8008E778093E80046
:1053400008952091E4003091E50095E64091EC004D
:10535000842F817040FF23C08091E80080FD1DC034
:1053600080919F02882399F0853099F08091EB001D
:1053700085FD11C04091E4005091E50024173507E8
:1053800029F3915011F09A01E1CF84E0089582E071
:10539000089583E0089581E0089580E008954091A4
:1053A000E80042FFDDCF08950E94422A0E944A2A67
:1053B000E0EEF0E0808181608083E8EDF0E08081C4
:1053C0008F77808319BCA7EDB0E08C918E7F8C9392
:1053D00080818F7E808310929E0208950F931F9389
:1053E000CF93DF930E94422A0E944A2AC8EDD0E060
:1053F00088818F77888388818068888388818F7D82
:10540000888319BC10929F0210929B0210929D02F9
:1054100010929C0200EE10E0F80180818B7F808367
:1054200088818160888342E060E080E00E944D29AD
:10543000E1EEF0E080818E7F8083E2EEF0E080811B
:1054400081608083808188608083F80180818E7F85
:105450008083888180618883DF91CF911F910F9134
:105460000895E8EDF0E080818F7E8083E7EDF0E045
:1054700080818160808384E082BF81E080939E028E
:105480000C94EE29E8EDF0E080818E7F808310920D
:10549000E20008951092DA001092E10008951F9240
:1054A0000F920FB60F9211242F933F934F935F9358
:1054B0006F937F938F939F93AF93BF93EF93FF93DC
:1054C0008091E10082FF0BC08091E20082FF07C063
:1054D0008091E1008B7F8093E1000E9412268091F1
:1054E000DA0080FF1FC08091D80080FF1BC0809130
:1054F000DA008E7F8093DA008091D90080FF0DC0A2
:1055000080E189BD82E189BD09B400FEFDCF81E063
:1055100080939F020E94D92505C019BC10929F025A
:105520000E94EB258091E10080FF19C08091E2008C
:1055300080FF15C08091E2008E7F8093E200809111
:10554000E20080618093E2008091D80080628093C5
:10555000D80019BC85E080939F020E94F8258091B5
:10556000E10084FF30C08091E20084FF2CC080E124
:1055700089BD82E189BD09B400FEFDCF8091D800CC
:105580008F7D8093D8008091E1008F7E8093E10031
:105590008091E2008F7E8093E2008091E200816042
:1055A0008093E20080919B02882311F084E007C081
:1055B0008091E30087FD02C081E001C083E0809319
:1055C0009F020E9404268091E10083FF29C0809100
:1055D000E20083FF25C08091E100877F8093E10096
:1055E00082E080939F0210929B028091E1008E7F67
:1055F0008093E1008091E2008E7F8093E2008091B1
:10560000E20080618093E20042E060E080E00E947E
:105610004D298091F00088608093F0000E94F2256F
:10562000FF91EF91BF91AF919F918F917F916F917A
:105630005F914F913F912F910F900FBE0F901F9050
:1056400018951F920F920FB60F9211242F933F932C
:105650004F935F936F937F938F939F93AF93BF937A
:10566000CF93DF93EF93FF93C091E900CF708091C8
:10567000EC00D82FD17080FDD0E81092E900809125
:10568000F000877F8093F00078940E94652B109241
:10569000E9008091F00088608093F000CD2BCF70FE
:1056A000C093E900FF91EF91DF91CF91BF91AF914E
:1056B0009F918F917F916F915F914F913F912F912A
:1056C0000F900FBE0F901F9018951F93CF93DF93ED
:1056D000CDB7DEB7AA970FB6F894DEBF0FBECDBF29
:1056E000E0EAF2E08091F100819322E0E83AF207EB
:1056F000C9F70E946C268091E80083FF2EC180913B
:10570000A0029091A102492F50E04A30510508F0C3
:1057100024C1FA01EE59FF4F0C94462D803821F038
:10572000823809F01AC108C080919C0290919D02B4
:10573000992389F082600FC08091A4028F70873016
:1057400008F00BC18093E9008091EB0085FB88276E
:1057500080F91092E9009091E800977F9093E8001B
:105760008093F1001092F100D1C0282F2D7F09F015
:10577000F4C0882319F0823061F0EFC08091A2025A
:10578000813009F0EAC0933009F080E080939D02F7
:105790002EC08091A20281112AC08091A4028F7034
:1057A0002FEF280F263008F0D8C08093E900209111
:1057B000EB0020FF1CC0933021F48091EB0080624D
:1057C00014C09091EB0090619093EB0021E030E0E9
:1057D000A90102C0440F551F8A95E2F74093EA00E1
:1057E0001092EA008091EB0088608093EB001092A9
:1057F000E9008091E800877F8093E8000E94822979
:10580000ACC08111AAC01091A2021F778091E30061
:105810008078812B8093E3008091E800877F8093DC
:10582000E8000E9482298091E80080FFFCCF8091EF
:10583000E30080688093E300111102C082E001C0A0
:1058400083E080939F0289C08058823008F085C031
:105850008091A2029091A3028C3D53E0950779F5C7
:1058600083E08A838AE289834FB7F894DE01139636
:1058700020E03EE051E2E32FF0E050935700E49146
:1058800020FF03C0E295EF703F5FEF708E2F90E036
:10589000EA3010F0C79601C0C0968D939D932F5F9C
:1058A000243149F74FBF8091E800877F8093E8005B
:1058B0006AE270E0CE0101960E948E2816C06091C7
:1058C000A4027091A502AE014F5F5F4F0E94D527E1
:1058D000BC01892B09F441C09091E800977F909317
:1058E000E80089819A810E94EC288091E8008B77FA
:1058F0008093E80032C0803881F58091E800877F8E
:105900008093E80080919B028093F1008091E800F1
:105910008E7772CF811121C08091A2029091A30253
:1059200099270297D4F48091E800877F8093E8005C
:105930008091A20280939B020E94822980919B0207
:10594000811106C08091E30087FD02C081E001C0A3
:1059500084E080939F020E9453268091E80083FF99
:105960000AC08091E800877F8093E8008091EB0077
:1059700080628093EB00AA960FB6F894DEBF0FBE4C
:10598000CDBFDF91CF911F910895CF9380919F025A
:105990008823A1F0C091E900CF709091EC00892F8D
:1059A000817090FD80E8C82B1092E9008091E8009A
:1059B00083FD0E94652BCF70C093E900CF910895BD
:1059C000DB018F939F930E945B2DBF91AF91A29FAC
:1059D000800D911DA39F900DB29F900D11240895ED
:1059E000991B79E004C0991F961708F0961B881F31
:1059F0007A95C9F780950895AA1BBB1B51E107C092
:105A0000AA1FBB1FA617B70710F0A61BB70B881F4E
:105A1000991F5A95A9F780959095BC01CD010895DD
:105A200097FB072E16F4009407D077FD09D00E944B
:105A3000FC2C07FC05D03EF4909581959F4F08956E
:105A4000709561957F4F0895A1E21A2EAA1BBB1B8A
:105A5000FD010DC0AA1FBB1FEE1FFF1FA217B3073A
:105A6000E407F50720F0A21BB30BE40BF50B661F50
:105A7000771F881F991F1A9469F760957095809514
:105A800090959B01AC01BD01CF010895EE0FFF1F62
:105A90000590F491E02D0994A29FB001B39FC0013D
:105AA000A39F700D811D1124911DB29F700D811D4A
:105AB0001124911D08950E944C2DA59F900DB49F17
:105AC000900DA49F800D911D11240895FB01DC0110
:105AD00004C08D910190801921F441505040C8F7C5
:105AE000881B990B0895F999FECF92BD81BDF89A54
:105AF000992780B50895A8E1B0E042E050E00C9409
:105B0000A72D262FF999FECF92BD81BDF89A019756
:105B100000B4021639F01FBA20BD0FB6F894FA9AF5
:105B2000F99A0FBE08950396272F0E94822D0E9496
:105B3000812D252F0E94822D242F0C94822D0196D9
:105B4000272F0E94822D0C94812DDC01CB01FC01BA
:105B5000F999FECF06C0F2BDE1BDF89A319600B4C6
:0E5B60000D9241505040B8F70895F894FFCFD1
:105B6E00C8004602280850011E0A140157257A253E
:105B7E005B25D525D1255A2501E200E900EA00B5BD
:105B8E0000B600B700CD008301CC008A01920194CB
:105B9E00012102230224022502260227022A02B331
:105BAE0000B4006F007000818283E200E900EA0019
:105BBE00B500B600B700CD008301CC008A0192017A
:105BCE0094012102230224022502260227022A0220
:105BDE00B300B4006F007000818283919094C697D9
:105BEE00663F3F3F006D6B5F64656C6179006D6B66
:105BFE005F696E74657276616C006D6B5F6D617856
:105C0E005F7370656564006D6B5F74696D655F745D
:105C1E006F5F6D6178006D6B5F776865656C5F6D4A
:105C2E0061785F7370656564006D6B5F776865653D
:105C3E006C5F74696D655F746F5F6D617800407B3A
:0E5C4E0022090B8E0A6C0A110A2A0A430A0068
:00000001FF
